 AsiBlCfg

 Timestamp is 57c98b3c (Fri Sep 02 10:22:52 2016)

 Preferred load address is 10000000

 Start         Length     Name                   Class
 0001:00000000 000045f4H .text$mn                CODE
 0001:00004600 0000002bH .text$x                 CODE
 0002:00000000 000001f0H .idata$5                DATA
 0002:000001f0 00000004H .CRT$XCA                DATA
 0002:000001f4 00000004H .CRT$XCZ                DATA
 0002:000001f8 00000004H .CRT$XIA                DATA
 0002:000001fc 00000004H .CRT$XIAA               DATA
 0002:00000200 00000004H .CRT$XIC                DATA
 0002:00000204 00000004H .CRT$XIZ                DATA
 0002:00000208 00000d08H .rdata                  DATA
 0002:00000f10 00000008H .rdata$sxdata           DATA
 0002:00000f18 00000004H .rtc$IAA                DATA
 0002:00000f1c 00000004H .rtc$IZZ                DATA
 0002:00000f20 00000004H .rtc$TAA                DATA
 0002:00000f24 00000004H .rtc$TZZ                DATA
 0002:00000f28 0000009cH .xdata$x                DATA
 0002:00000fd0 000000bdH .edata                  DATA
 0002:00001090 000000a0H .idata$2                DATA
 0002:00001130 00000014H .idata$3                DATA
 0002:00001144 000001f0H .idata$4                DATA
 0002:00001334 000008f6H .idata$6                DATA
 0003:00000000 0000050cH .data                   DATA
 0003:00000510 00000430H .bss                    DATA
 0004:00000000 000002c8H .rsrc$01                DATA
 0004:000002d0 0002cb88H .rsrc$02                DATA

  Address         Publics by Value              Rva+Base       Lib:Object

 0000:00000000       ___guard_fids_count        00000000     <absolute>
 0000:00000000       ___guard_fids_table        00000000     <absolute>
 0000:00000000       ___guard_flags             00000000     <absolute>
 0000:00000002       ___safe_se_handler_count   00000002     <absolute>
 0000:00000000       ___ImageBase               10000000     <linker-defined>
 0001:00000000       ?IsSectionPresent@ControlPanelRegistration@@AAE_NPAUreg_list@@@Z 10001000 f   CtrlPnlReg.obj
 0001:00000090       ?AddList@ControlPanelRegistration@@AAE_NPAUkey_path_entry@@PAUreg_list_entry@@@Z 10001090 f   CtrlPnlReg.obj
 0001:000001d0       ?AddSection@ControlPanelRegistration@@AAE_NPAUreg_list@@@Z 100011d0 f   CtrlPnlReg.obj
 0001:00000250       ?RemoveList@ControlPanelRegistration@@AAE_NPAUkey_path_entry@@PAUreg_list_entry@@@Z 10001250 f   CtrlPnlReg.obj
 0001:00000360       ?FindValueName@ControlPanelRegistration@@AAE_NPAUHKEY__@@PB_WPA_WH@Z 10001360 f   CtrlPnlReg.obj
 0001:00000420       ?FindFirstOpenEntry@ControlPanelRegistration@@AAEXPAUHKEY__@@PA_W@Z 10001420 f   CtrlPnlReg.obj
 0001:00000470       ?Register@ControlPanelRegistration@@QAE_NXZ 10001470 f   CtrlPnlReg.obj
 0001:00000560       ?UnRegister@ControlPanelRegistration@@QAE_NXZ 10001560 f   CtrlPnlReg.obj
 0001:00000660       ?Show@ControlPanelRegistration@@QAE_N_N@Z 10001660 f   CtrlPnlReg.obj
 0001:00000760       ?SetChannel@BluLinkChannelControl@@QAEXH@Z 10001760 f i AdapterInfo.obj
 0001:00000840       ?GetColor@BluLinkChannelControl@@QAEKXZ 10001840 f i AdapterInfo.obj
 0001:00000870       ?SetChannelsPerDevice@DialogParameters@@QAEXH@Z 10001870 f i AdapterInfo.obj
 0001:000008e0       ?AllocateBlulinkControls@DialogParameters@@QAEXXZ 100018e0 f i AdapterInfo.obj
 0001:00000a20       ??_H@YGXPAXIHP6EPAX0@Z@Z   10001a20 f i AdapterInfo.obj
 0001:00000a60       ?set_flag@quick_conflict_detector@@QAEXK@Z 10001a60 f i AdapterInfo.obj
 0001:00000b00       ?GetChannelFromHpiControl@@YAHII@Z 10001b00 f   AdapterInfo.obj
 0001:00000c20       ?InitChannelCount@AsiBluLinkConfigPerAdapterInfo@@QAEXPAVDialogParameters@@PAX@Z 10001c20 f   AdapterInfo.obj
 0001:00000cc0       ?InitChannels@AsiBluLinkConfigPerAdapterInfo@@QAEXPAVDialogParameters@@PAX@Z 10001cc0 f   AdapterInfo.obj
 0001:00000ed0       ?ReportHpiError@@YAXPB_WG@Z 10001ed0 f   AdapterInfo.obj
 0001:00000f10       ?SaveChannelToHpiControl@@YAXIIH@Z 10001f10 f   AdapterInfo.obj
 0001:000010d0       ?SaveChannels@AsiBluLinkConfigPerAdapterInfo@@QAEXPAVDialogParameters@@PAX@Z 100020d0 f   AdapterInfo.obj
 0001:00001290       ?FoundAsiRegistryKey@AsiBluLinkConfigAdapterInfo@@AAEHPAVDialogParameters@@PAUHKEY__@@@Z 10002290 f   AdapterInfo.obj
 0001:00001370       ?InitChannelsPerDevice@AsiBluLinkConfigAdapterInfo@@AAEXPAVDialogParameters@@PAUHWND__@@@Z 10002370 f   AdapterInfo.obj
 0001:00001540       ?InitAdapterInfo@AsiBluLinkConfigAdapterInfo@@QAEHPAVDialogParameters@@PAUHWND__@@_N@Z 10002540 f   AdapterInfo.obj
 0001:00001880       ?SaveAdapterInfo@AsiBluLinkConfigAdapterInfo@@QAEXPAVDialogParameters@@_N@Z 10002880 f   AdapterInfo.obj
 0001:000019b0       ?CountBluPciAdapters@@YAHPAH@Z 100029b0 f   AdapterInfo.obj
 0001:00001a50       _DllMain@12                10002a50 f   BluLinkCfg.obj
 0001:00001a80       ?ShowControlPanel_RunDll@@YGXPAUHWND__@@PAUHINSTANCE__@@PADH@Z 10002a80 f   BluLinkCfg.obj
 0001:00001b40       ?RegisterControlPanelApplet_RunDll@@YGXPAUHWND__@@PAUHINSTANCE__@@PADH@Z 10002b40 f   BluLinkCfg.obj
 0001:00001c30       ?DllRegisterServer@@YGJXZ  10002c30 f   BluLinkCfg.obj
 0001:00001cf0       ?DllUnregisterServer@@YGJXZ 10002cf0 f   BluLinkCfg.obj
 0001:00001d60       ?SetConflict@BluLinkChannelControl@@QAEXPAV1@@Z 10002d60 f i ChanControl.obj
 0001:00001dd0       ?ReplaceBackgroundColor@@YAXPAUHWND__@@K@Z 10002dd0 f   ChanControl.obj
 0001:00001eb0       ?BluLinkChannelEditSubclassProc@@YGJPAUHWND__@@IIJIK@Z 10002eb0 f   ChanControl.obj
 0001:00002110       ??0DialogParameters@@QAE@_N@Z 10003110 f i ConfigDialog.obj
 0001:000021b0       ??1DialogParameters@@QAE@XZ 100031b0 f i ConfigDialog.obj
 0001:00002200       ?AnyConflicts@DialogParameters@@QAE_NXZ 10003200 f i ConfigDialog.obj
 0001:00002230       ??1AsiBluLinkConfigAdapterInfo@@QAE@XZ 10003230 f i ConfigDialog.obj
 0001:000022a0       ?KeyboardProc@KeyboardHook@@CGJHIJ@Z 100032a0 f   ConfigDialog.obj
 0001:00002330       ?CheckInitialSettings@DialogParameters@@QAEXPAUHWND__@@@Z 10003330 f   ConfigDialog.obj
 0001:00002520       ?CreateGroupOfControls@DialogParameters@@QAEPAGPAGHHKKK@Z 10003520 f   ConfigDialog.obj
 0001:00002670       ?CustomizeDialog@DialogParameters@@QAEPAEPAEH@Z 10003670 f   ConfigDialog.obj
 0001:00002900       ?CheckTxConflicts@DialogParameters@@QAEXPAVBluLinkChannelControl@@@Z 10003900 f   ConfigDialog.obj
 0001:00002a10       ?RunRebootDialog@DialogParameters@@QAEHPAUHWND__@@@Z 10003a10 f   ConfigDialog.obj
 0001:00002b20       ?CheckSampleRateMismatch@DialogParameters@@QAEHPAUHWND__@@@Z 10003b20 f   ConfigDialog.obj
 0001:00002cb0       ?GuiSamplerateChange@DialogParameters@@QAEXPAUHWND__@@H@Z 10003cb0 f   ConfigDialog.obj
 0001:00002e20       ??0AsiScrollbar@@QAE@PAUHWND__@@HHH@Z 10003e20 f i ConfigDialog.obj
 0001:00002ec0       ?HandleScrollMessage@AsiScrollbar@@QAEXGG@Z 10003ec0 f i ConfigDialog.obj
 0001:00003000       ?InitControls@@YAXPAUHWND__@@PAVDialogParameters@@@Z 10004000 f   ConfigDialog.obj
 0001:000034e0       ?CalculateMaxScroll@@YAHPAUHWND__@@@Z 100044e0 f   ConfigDialog.obj
 0001:00003550       ?SetChannelValue@@YAXPAUHWND__@@PAVBluLinkChannelControl@@PAVDialogParameters@@IH@Z 10004550 f   ConfigDialog.obj
 0001:000035d0       ?EditControlMessage@@YAHPAUHWND__@@IJPAVDialogParameters@@@Z 100045d0 f   ConfigDialog.obj
 0001:00003730       ?DialogProc@@YGHPAUHWND__@@IIJ@Z 10004730 f   ConfigDialog.obj
 0001:00003a80       ?SetControlToBold@@YAXPAUHWND__@@H@Z 10004a80 f   ConfigDialog.obj
 0001:00003b50       ?RebootDialogProc@@YGHPAUHWND__@@IIJ@Z 10004b50 f   ConfigDialog.obj
 0001:00003c00       ?RunDialog@@YAXPAUHWND__@@_N@Z 10004c00 f   ConfigDialog.obj
 0001:00003d06       @__security_check_cookie@4 10004d06 f   MSVCRT:secchk.obj
 0001:00003d61       __CRT_INIT@12              10004d61 f   MSVCRT:crtdll.obj
 0001:00003f58       __DllMainCRTStartup@12     10004f58 f   MSVCRT:crtdll.obj
 0001:000040ae       ___raise_securityfailure   100050ae f   MSVCRT:gs_report.obj
 0001:000040eb       ___report_gsfailure        100050eb f   MSVCRT:gs_report.obj
 0001:000041e6       ___CppXcptFilter           100051e6 f   MSVCRT:MSVCR120.dll
 0001:000041ec       __amsg_exit                100051ec f   MSVCRT:MSVCR120.dll
 0001:00004200       __FindPESection            10005200 f   MSVCRT:pesect.obj
 0001:00004250       __IsNonwritableInCurrentImage 10005250 f   MSVCRT:pesect.obj
 0001:00004310       __ValidateImageBase        10005310 f   MSVCRT:pesect.obj
 0001:00004341       ___atonexitinit            10005341 f   MSVCRT:atonexit.obj
 0001:0000437d       __onexit                   1000537d f   MSVCRT:atonexit.obj
 0001:00004426       _atexit                    10005426 f   MSVCRT:atonexit.obj
 0001:0000443b       ___security_init_cookie    1000543b f   MSVCRT:gs_support.obj
 0001:000044d7       __RTC_Initialize           100054d7 f   MSVCRT:initsect.obj
 0001:000044f7       __RTC_Terminate            100054f7 f   MSVCRT:initsect.obj
 0001:00004518       __initterm                 10005518 f   MSVCRT:MSVCR120.dll
 0001:0000451e       __initterm_e               1000551e f   MSVCRT:MSVCR120.dll
 0001:00004524       ___clean_type_info_names   10005524 f   MSVCRT:tncleanup.obj
 0001:00004530       __SEH_prolog4              10005530 f   MSVCRT:sehprolg4.obj
 0001:00004575       __SEH_epilog4              10005575 f   MSVCRT:sehprolg4.obj
 0001:00004589       __except_handler4          10005589 f   MSVCRT:chandler4gs.obj
 0001:000045ac       __crt_debugger_hook        100055ac f   MSVCRT:MSVCR120.dll
 0001:000045b2       ___crtUnhandledException   100055b2 f   MSVCRT:MSVCR120.dll
 0001:000045b8       ___crtTerminateProcess     100055b8 f   MSVCRT:MSVCR120.dll
 0001:000045be       __lock                     100055be f   MSVCRT:MSVCR120.dll
 0001:000045c4       __unlock                   100055c4 f   MSVCRT:MSVCR120.dll
 0001:000045ca       ___dllonexit               100055ca f   MSVCRT:MSVCR120.dll
 0001:000045d0       ___clean_type_info_names_internal 100055d0 f   MSVCRT:MSVCR120.dll
 0001:000045d6       __except_handler4_common   100055d6 f   MSVCRT:MSVCR120.dll
 0001:000045dc       _IsProcessorFeaturePresent@4 100055dc f   kernel32:KERNEL32.dll
 0001:000045e2       ___CxxFrameHandler3        100055e2 f   MSVCRT:MSVCR120.dll
 0001:000045e8       _memcpy                    100055e8 f   MSVCRT:MSVCR120.dll
 0001:000045ee       _memset                    100055ee f   MSVCRT:MSVCR120.dll
 0002:00000000       __imp__RegDeleteValueW@8   10006000     advapi32:ADVAPI32.dll
 0002:00000004       __imp__AdjustTokenPrivileges@24 10006004     advapi32:ADVAPI32.dll
 0002:00000008       __imp__LookupPrivilegeValueW@12 10006008     advapi32:ADVAPI32.dll
 0002:0000000c       __imp__RegDeleteKeyW@8     1000600c     advapi32:ADVAPI32.dll
 0002:00000010       __imp__RegQueryValueExW@24 10006010     advapi32:ADVAPI32.dll
 0002:00000014       __imp__RegCreateKeyExW@36  10006014     advapi32:ADVAPI32.dll
 0002:00000018       __imp__RegEnumValueW@32    10006018     advapi32:ADVAPI32.dll
 0002:0000001c       __imp__RegOpenKeyExW@20    1000601c     advapi32:ADVAPI32.dll
 0002:00000020       __imp__OpenProcessToken@12 10006020     advapi32:ADVAPI32.dll
 0002:00000024       __imp__RegSetValueExW@24   10006024     advapi32:ADVAPI32.dll
 0002:00000028       __imp__RegCloseKey@4       10006028     advapi32:ADVAPI32.dll
 0002:0000002c       \177ADVAPI32_NULL_THUNK_DATA 1000602c     advapi32:ADVAPI32.dll
 0002:00000030       __imp__HPI_Object_GetValueEntity@8 10006030     asihpi32:ASIHPI32.dll
 0002:00000034       __imp__HPI_Entity_Unpack@20 10006034     asihpi32:ASIHPI32.dll
 0002:00000038       __imp__HPI_Entity_Free@4   10006038     asihpi32:ASIHPI32.dll
 0002:0000003c       __imp__HPI_AdapterGetProperty@20 1000603c     asihpi32:ASIHPI32.dll
 0002:00000040       __imp__HPI_Object_GetInfo@24 10006040     asihpi32:ASIHPI32.dll
 0002:00000044       __imp__HPI_Entity_AllocAndPack@24 10006044     asihpi32:ASIHPI32.dll
 0002:00000048       __imp__HPI_Universal_Set@12 10006048     asihpi32:ASIHPI32.dll
 0002:0000004c       __imp__HPI_SubSysGetAdapter@16 1000604c     asihpi32:ASIHPI32.dll
 0002:00000050       __imp__HPI_AdapterOpen@8   10006050     asihpi32:ASIHPI32.dll
 0002:00000054       __imp__HPI_MixerOpen@12    10006054     asihpi32:ASIHPI32.dll
 0002:00000058       __imp__HPI_MixerClose@8    10006058     asihpi32:ASIHPI32.dll
 0002:0000005c       __imp__HPI_AdapterClose@8  1000605c     asihpi32:ASIHPI32.dll
 0002:00000060       __imp__HPI_SubSysCreate@0  10006060     asihpi32:ASIHPI32.dll
 0002:00000064       __imp__HPI_SubSysGetNumAdapters@8 10006064     asihpi32:ASIHPI32.dll
 0002:00000068       __imp__HPI_Object_ParameterHandle@16 10006068     asihpi32:ASIHPI32.dll
 0002:0000006c       __imp__HPI_SampleClock_GetLocalRate@12 1000606c     asihpi32:ASIHPI32.dll
 0002:00000070       __imp__HPI_MixerGetControl@32 10006070     asihpi32:ASIHPI32.dll
 0002:00000074       __imp__HPI_SampleClock_SetLocalRate@12 10006074     asihpi32:ASIHPI32.dll
 0002:00000078       \177ASIHPI32_NULL_THUNK_DATA 10006078     asihpi32:ASIHPI32.dll
 0002:0000007c       __imp__SetWindowSubclass@16 1000607c     Comctl32:COMCTL32.dll
 0002:00000080       __imp__DefSubclassProc@16  10006080     Comctl32:COMCTL32.dll
 0002:00000084       \177COMCTL32_NULL_THUNK_DATA 10006084     Comctl32:COMCTL32.dll
 0002:00000088       __imp__CreateSolidBrush@4  10006088     gdi32:GDI32.dll
 0002:0000008c       __imp__BitBlt@36           1000608c     gdi32:GDI32.dll
 0002:00000090       __imp__GetTextMetricsW@8   10006090     gdi32:GDI32.dll
 0002:00000094       __imp__GetTextFaceW@12     10006094     gdi32:GDI32.dll
 0002:00000098       __imp__CreateFontIndirectW@4 10006098     gdi32:GDI32.dll
 0002:0000009c       __imp__SelectObject@8      1000609c     gdi32:GDI32.dll
 0002:000000a0       \177GDI32_NULL_THUNK_DATA  100060a0     gdi32:GDI32.dll
 0002:000000a4       __imp__DecodePointer@4     100060a4     kernel32:KERNEL32.dll
 0002:000000a8       __imp__IsDebuggerPresent@0 100060a8     kernel32:KERNEL32.dll
 0002:000000ac       __imp__IsProcessorFeaturePresent@4 100060ac     kernel32:KERNEL32.dll
 0002:000000b0       __imp__GetLastError@0      100060b0     kernel32:KERNEL32.dll
 0002:000000b4       __imp__EncodePointer@4     100060b4     kernel32:KERNEL32.dll
 0002:000000b8       __imp__GlobalFree@4        100060b8     kernel32:KERNEL32.dll
 0002:000000bc       __imp__GetCurrentProcessId@0 100060bc     kernel32:KERNEL32.dll
 0002:000000c0       __imp__QueryPerformanceCounter@4 100060c0     kernel32:KERNEL32.dll
 0002:000000c4       __imp__DisableThreadLibraryCalls@4 100060c4     kernel32:KERNEL32.dll
 0002:000000c8       __imp__GetProcAddress@8    100060c8     kernel32:KERNEL32.dll
 0002:000000cc       __imp__GetModuleHandleW@4  100060cc     kernel32:KERNEL32.dll
 0002:000000d0       __imp__GetCurrentProcess@0 100060d0     kernel32:KERNEL32.dll
 0002:000000d4       __imp__GetCurrentThreadId@0 100060d4     kernel32:KERNEL32.dll
 0002:000000d8       __imp__GlobalAlloc@8       100060d8     kernel32:KERNEL32.dll
 0002:000000dc       __imp__GetSystemTimeAsFileTime@4 100060dc     kernel32:KERNEL32.dll
 0002:000000e0       \177KERNEL32_NULL_THUNK_DATA 100060e0     kernel32:KERNEL32.dll
 0002:000000e4       __imp____CppXcptFilter     100060e4     MSVCRT:MSVCR120.dll
 0002:000000e8       __imp___vswprintf_c_l      100060e8     MSVCRT:MSVCR120.dll
 0002:000000ec       __imp_??2@YAPAXI@Z         100060ec     MSVCRT:MSVCR120.dll
 0002:000000f0       __imp_??3@YAXPAX@Z         100060f0     MSVCRT:MSVCR120.dll
 0002:000000f4       __imp___swprintf           100060f4     MSVCRT:MSVCR120.dll
 0002:000000f8       __imp__memset              100060f8     MSVCRT:MSVCR120.dll
 0002:000000fc       __imp___wcsicmp            100060fc     MSVCRT:MSVCR120.dll
 0002:00000100       __imp___amsg_exit          10006100     MSVCRT:MSVCR120.dll
 0002:00000104       __imp__free                10006104     MSVCRT:MSVCR120.dll
 0002:00000108       __imp___malloc_crt         10006108     MSVCRT:MSVCR120.dll
 0002:0000010c       __imp___initterm           1000610c     MSVCRT:MSVCR120.dll
 0002:00000110       __imp___initterm_e         10006110     MSVCRT:MSVCR120.dll
 0002:00000114       __imp___crt_debugger_hook  10006114     MSVCRT:MSVCR120.dll
 0002:00000118       __imp____crtUnhandledException 10006118     MSVCRT:MSVCR120.dll
 0002:0000011c       __imp____crtTerminateProcess 1000611c     MSVCRT:MSVCR120.dll
 0002:00000120       __imp___lock               10006120     MSVCRT:MSVCR120.dll
 0002:00000124       __imp___unlock             10006124     MSVCRT:MSVCR120.dll
 0002:00000128       __imp___calloc_crt         10006128     MSVCRT:MSVCR120.dll
 0002:0000012c       __imp____dllonexit         1000612c     MSVCRT:MSVCR120.dll
 0002:00000130       __imp___onexit             10006130     MSVCRT:MSVCR120.dll
 0002:00000134       __imp___except_handler4_common 10006134     MSVCRT:MSVCR120.dll
 0002:00000138       __imp__exit                10006138     MSVCRT:MSVCR120.dll
 0002:0000013c       __imp____CxxFrameHandler3  1000613c     MSVCRT:MSVCR120.dll
 0002:00000140       __imp__memcpy              10006140     MSVCRT:MSVCR120.dll
 0002:00000144       __imp____clean_type_info_names_internal 10006144     MSVCRT:MSVCR120.dll
 0002:00000148       \177MSVCR120_NULL_THUNK_DATA 10006148     MSVCRT:MSVCR120.dll
 0002:0000014c       __imp__SetupDiGetClassDevsW@16 1000614c     Setupapi:SETUPAPI.dll
 0002:00000150       __imp__SetupDiOpenDevRegKey@24 10006150     Setupapi:SETUPAPI.dll
 0002:00000154       __imp__SetupDiDestroyDeviceInfoList@4 10006154     Setupapi:SETUPAPI.dll
 0002:00000158       __imp__SetupDiEnumDeviceInfo@12 10006158     Setupapi:SETUPAPI.dll
 0002:0000015c       \177SETUPAPI_NULL_THUNK_DATA 1000615c     Setupapi:SETUPAPI.dll
 0002:00000160       __imp__SetWindowLongW@12   10006160     user32:USER32.dll
 0002:00000164       __imp__SetWindowPos@28     10006164     user32:USER32.dll
 0002:00000168       __imp__GetWindowLongW@8    10006168     user32:USER32.dll
 0002:0000016c       __imp__GetDlgItemInt@16    1000616c     user32:USER32.dll
 0002:00000170       __imp__SetDlgItemInt@16    10006170     user32:USER32.dll
 0002:00000174       __imp__SetDlgItemTextW@12  10006174     user32:USER32.dll
 0002:00000178       __imp__SetWindowTextW@8    10006178     user32:USER32.dll
 0002:0000017c       __imp__ShowWindow@8        1000617c     user32:USER32.dll
 0002:00000180       __imp__ScrollWindowEx@32   10006180     user32:USER32.dll
 0002:00000184       __imp__ClientToScreen@8    10006184     user32:USER32.dll
 0002:00000188       __imp__SetScrollInfo@16    10006188     user32:USER32.dll
 0002:0000018c       __imp__EndDialog@8         1000618c     user32:USER32.dll
 0002:00000190       __imp__SendDlgItemMessageW@20 10006190     user32:USER32.dll
 0002:00000194       __imp__EnableWindow@8      10006194     user32:USER32.dll
 0002:00000198       __imp__CheckRadioButton@16 10006198     user32:USER32.dll
 0002:0000019c       __imp__DialogBoxParamW@20  1000619c     user32:USER32.dll
 0002:000001a0       __imp__GetWindowRect@8     100061a0     user32:USER32.dll
 0002:000001a4       __imp__GetDesktopWindow@0  100061a4     user32:USER32.dll
 0002:000001a8       __imp__GetDlgItem@8        100061a8     user32:USER32.dll
 0002:000001ac       __imp__IsWindowEnabled@4   100061ac     user32:USER32.dll
 0002:000001b0       __imp__CallNextHookEx@16   100061b0     user32:USER32.dll
 0002:000001b4       __imp__SendInput@12        100061b4     user32:USER32.dll
 0002:000001b8       __imp__UnhookWindowsHookEx@4 100061b8     user32:USER32.dll
 0002:000001bc       __imp__SetWindowsHookExW@16 100061bc     user32:USER32.dll
 0002:000001c0       __imp__ReleaseDC@8         100061c0     user32:USER32.dll
 0002:000001c4       __imp__GetDC@4             100061c4     user32:USER32.dll
 0002:000001c8       __imp__SendMessageW@16     100061c8     user32:USER32.dll
 0002:000001cc       __imp__MessageBoxW@16      100061cc     user32:USER32.dll
 0002:000001d0       __imp__InvalidateRect@12   100061d0     user32:USER32.dll
 0002:000001d4       __imp__GetClientRect@8     100061d4     user32:USER32.dll
 0002:000001d8       __imp__IsDlgButtonChecked@8 100061d8     user32:USER32.dll
 0002:000001dc       __imp__LoadStringW@16      100061dc     user32:USER32.dll
 0002:000001e0       __imp__DialogBoxIndirectParamW@20 100061e0     user32:USER32.dll
 0002:000001e4       __imp__ExitWindowsEx@8     100061e4     user32:USER32.dll
 0002:000001e8       __imp__ScreenToClient@8    100061e8     user32:USER32.dll
 0002:000001ec       \177USER32_NULL_THUNK_DATA 100061ec     user32:USER32.dll
 0002:000001f0       ___xc_a                    100061f0     MSVCRT:cinitexe.obj
 0002:000001f4       ___xc_z                    100061f4     MSVCRT:cinitexe.obj
 0002:000001f8       ___xi_a                    100061f8     MSVCRT:cinitexe.obj
 0002:00000204       ___xi_z                    10006204     MSVCRT:cinitexe.obj
 0002:00000208       _GUID_DEVCLASS_MEDIA       10006208     uuid:cguid_i.obj
 0002:00000218       __pRawDllMain              10006218     MSVCRT:crtdll.obj
 0002:00000218       __pDefaultRawDllMain       10006218     MSVCRT:crtdll.obj
 0002:00000224       ??_C@_1BI@IDMJHIIF@?$AAD?$AAe?$AAf?$AAa?$AAu?$AAl?$AAt?$AAI?$AAc?$AAo?$AAn?$AA?$AA@ 10006224     CtrlPnlReg.obj
 0002:0000023c       ??_C@_1M@JLDCNMKN@?$AAS?$AAh?$AAe?$AAl?$AAl?$AA?$AA@ 1000623c     CtrlPnlReg.obj
 0002:00000248       ??_C@_1BA@MGKEIBAA@?$AAC?$AAo?$AAm?$AAm?$AAa?$AAn?$AAd?$AA?$AA@ 10006248     CtrlPnlReg.obj
 0002:00000258       ??_C@_1CA@KMFDEJAN@?$AAL?$AAo?$AAc?$AAa?$AAl?$AAi?$AAz?$AAe?$AAd?$AAS?$AAt?$AAr?$AAi?$AAn?$AAg?$AA?$AA@ 10006258     CtrlPnlReg.obj
 0002:00000278       ??_C@_1BA@NFCMADAA@?$AAI?$AAn?$AAf?$AAo?$AAT?$AAi?$AAp?$AA?$AA@ 10006278     CtrlPnlReg.obj
 0002:00000288       ??_C@_1CO@MIJIOHLE@?$AAS?$AAy?$AAs?$AAt?$AAe?$AAm?$AA?4?$AAA?$AAp?$AAp?$AAl?$AAi?$AAc?$AAa?$AAt?$AAi?$AAo?$AAn?$AAN?$AAa?$AAm?$AAe?$AA?$AA@ 10006288     CtrlPnlReg.obj
 0002:000002b8       ??_C@_1DK@DDDACLHP@?$AAS?$AAy?$AAs?$AAt?$AAe?$AAm?$AA?4?$AAC?$AAo?$AAn?$AAt?$AAr?$AAo?$AAl?$AAP?$AAa?$AAn?$AAe?$AAl?$AA?4?$AAC?$AAa?$AAt?$AAe?$AAg?$AAo?$AAr?$AAy?$AA?$AA@ 100062b8     CtrlPnlReg.obj
 0002:000002f4       ??_C@_1M@KANJNLFF@?$AAC?$AAL?$AAS?$AAI?$AAD?$AA?$AA@ 100062f4     CtrlPnlReg.obj
 0002:00000300       ??_C@_1JE@KFOKPFDN@?$AAS?$AAO?$AAF?$AAT?$AAW?$AAA?$AAR?$AAE?$AA?2?$AAM?$AAi?$AAc?$AAr?$AAo?$AAs?$AAo?$AAf?$AAt?$AA?2?$AAW?$AAi?$AAn?$AAd?$AAo?$AAw?$AAs?$AA?2?$AAC?$AAu?$AAr?$AAr?$AAe@ 10006300     CtrlPnlReg.obj
 0002:00000394       ??_C@_1BC@PKEHKAEB@?$AAE?$AAx?$AAp?$AAl?$AAo?$AAr?$AAe?$AAr?$AA?$AA@ 10006394     CtrlPnlReg.obj
 0002:000003a8       ??_C@_1BI@DMHEGHBF@?$AAD?$AAi?$AAs?$AAa?$AAl?$AAl?$AAo?$AAw?$AAC?$AAp?$AAl?$AA?$AA@ 100063a8     CtrlPnlReg.obj
 0002:000003c0       ??_C@_1GG@IPMCGENI@?$AAS?$AAO?$AAF?$AAT?$AAW?$AAA?$AAR?$AAE?$AA?2?$AAM?$AAi?$AAc?$AAr?$AAo?$AAs?$AAo?$AAf?$AAt?$AA?2?$AAW?$AAi?$AAn?$AAd?$AAo?$AAw?$AAs?$AA?2?$AAC?$AAu?$AAr?$AAr?$AAe@ 100063c0     CtrlPnlReg.obj
 0002:00000428       ??_C@_15KNBIKKIN@?$AA?$CF?$AAd?$AA?$AA@ 10006428     CtrlPnlReg.obj
 0002:00000430       ??_C@_1M@DMOFNHON@?$AAR?$AAu?$AAn?$AAA?$AAs?$AA?$AA@ 10006430     CtrlPnlReg.obj
 0002:00000440       ??_C@_1JA@EMBPJHGA@?$AAS?$AAO?$AAF?$AAT?$AAW?$AAA?$AAR?$AAE?$AA?2?$AAM?$AAi?$AAc?$AAr?$AAo?$AAs?$AAo?$AAf?$AAt?$AA?2?$AAW?$AAi?$AAn?$AAd?$AAo?$AAw?$AAs?$AA?2?$AAC?$AAu?$AAr?$AAr?$AAe@ 10006440     CtrlPnlReg.obj
 0002:000004d4       ?m_initial_count@quick_conflict_detector@@0HB 100064d4     AdapterInfo.obj
 0002:000004d8       ?m_bits_per_entry@quick_conflict_detector@@0HB 100064d8     AdapterInfo.obj
 0002:000004dc       ??_C@_1CK@PCFIAPBJ@?$AAC?$AAh?$AAa?$AAn?$AAn?$AAe?$AAl?$AAs?$AAP?$AAe?$AAr?$AAS?$AAu?$AAb?$AAd?$AAe?$AAv?$AAi?$AAc?$AAe?$AA?$AA@ 100064dc     AdapterInfo.obj
 0002:00000508       ??_C@_07DMJBFPJJ@Channel?$AA@ 10006508     AdapterInfo.obj
 0002:00000510       ??_C@_1DG@LNIOOGGI@?$AAH?$AAP?$AAI?$AA_?$AAO?$AAb?$AAj?$AAe?$AAc?$AAt?$AA_?$AAP?$AAa?$AAr?$AAa?$AAm?$AAe?$AAt?$AAe?$AAr?$AAH?$AAa?$AAn?$AAd?$AAl?$AAe?$AA?$AA@ 10006510     AdapterInfo.obj
 0002:00000548       ??_C@_1EE@PDNLGPFH@?$AAF?$AAu?$AAn?$AAc?$AAt?$AAi?$AAo?$AAn?$AA?3?$AA?5?$AA?$CC?$AA?$CF?$AAs?$AA?$CC?$AA?5?$AAr?$AAe?$AAt?$AAu?$AAr?$AAn?$AAe?$AAd?$AA?5?$AAe?$AAr?$AAr?$AAo?$AAr?$AA?3?$AA?5?$AA?$CF@ 10006548     AdapterInfo.obj
 0002:0000058c       ??_C@_1CG@EPCCAABM@?$AAH?$AAP?$AAI?$AA_?$AAO?$AAb?$AAj?$AAe?$AAc?$AAt?$AA_?$AAG?$AAe?$AAt?$AAI?$AAn?$AAf?$AAo?$AA?$AA@ 1000658c     AdapterInfo.obj
 0002:000005b4       ??_C@_1CK@OJGCMPLE@?$AAe?$AAn?$AAt?$AAi?$AAt?$AAy?$AA?5?$AAn?$AAo?$AAt?$AA?5?$AAw?$AAr?$AAi?$AAt?$AAe?$AAa?$AAb?$AAl?$AAe?$AA?$AA@ 100065b4     AdapterInfo.obj
 0002:000005e0       ??_C@_1DE@CHMJBILK@?$AAH?$AAP?$AAI?$AA_?$AAO?$AAb?$AAj?$AAe?$AAc?$AAt?$AA_?$AAG?$AAe?$AAt?$AAV?$AAa?$AAl?$AAu?$AAe?$AAE?$AAn?$AAt?$AAi?$AAt?$AAy?$AA?$AA@ 100065e0     AdapterInfo.obj
 0002:00000614       ??_C@_1CE@IIDJKCDC@?$AAH?$AAP?$AAI?$AA_?$AAU?$AAn?$AAi?$AAv?$AAe?$AAr?$AAs?$AAa?$AAl?$AA_?$AAS?$AAe?$AAt?$AA?$AA@ 10006614     AdapterInfo.obj
 0002:00000638       ??_C@_1DA@MIHDLDAM@?$AAH?$AAP?$AAI?$AA_?$AAE?$AAn?$AAt?$AAi?$AAt?$AAy?$AA_?$AAA?$AAl?$AAl?$AAo?$AAc?$AAA?$AAn?$AAd?$AAP?$AAa?$AAc?$AAk?$AA?$AA@ 10006638     AdapterInfo.obj
 0002:00000668       ??_C@_1CA@BDNGJNOP@?$AAt?$AAy?$AAp?$AAe?$AA?5?$AAi?$AAs?$AA?5?$AAn?$AAo?$AAt?$AA?5?$AAi?$AAn?$AAt?$AA?$AA@ 10006668     AdapterInfo.obj
 0002:00000688       ??_C@_1CA@DLBCANMK@?$AAH?$AAP?$AAI?$AAA?$AAd?$AAa?$AAp?$AAt?$AAe?$AAr?$AAI?$AAn?$AAd?$AAe?$AAx?$AA?$AA@ 10006688     AdapterInfo.obj
 0002:000006a8       ??_C@_1O@GAOCKAOK@?$AAD?$AAr?$AAi?$AAv?$AAe?$AAr?$AA?$AA@ 100066a8     AdapterInfo.obj
 0002:000006b8       ??_C@_1BK@CJIHEDPJ@?$AAa?$AAs?$AAi?$AAw?$AAd?$AAm?$AAx?$AAv?$AA?4?$AAs?$AAy?$AAs?$AA?$AA@ 100066b8     AdapterInfo.obj
 0002:000006d4       ??_C@_1BK@HPPNMIOH@?$AAa?$AAs?$AAi?$AAw?$AAd?$AAm?$AA6?$AA4?$AA?4?$AAs?$AAy?$AAs?$AA?$AA@ 100066d4     AdapterInfo.obj
 0002:000006f0       ??_C@_1BK@EAIFNPAP@?$AAA?$AAs?$AAi?$AAB?$AAl?$AAC?$AAf?$AAg?$AA?4?$AAd?$AAl?$AAl?$AA?$AA@ 100066f0     BluLinkCfg.obj
 0002:00000710       ??_C@_1II@HHFPHICK@?$AAr?$AAu?$AAn?$AAd?$AAl?$AAl?$AA3?$AA2?$AA?5?$AA?$CF?$AAS?$AAy?$AAs?$AAt?$AAe?$AAm?$AAR?$AAo?$AAo?$AAt?$AA?$CF?$AA?2?$AAs?$AAy?$AAs?$AAt?$AAe?$AAm?$AA3?$AA2?$AA?2?$AAA@ 10006710     BluLinkCfg.obj
 0002:00000798       ??_C@_1FA@CLEABNMM@?$AA?$CF?$AAS?$AAy?$AAs?$AAt?$AAe?$AAm?$AAR?$AAo?$AAo?$AAt?$AA?$CF?$AA?2?$AAs?$AAy?$AAs?$AAt?$AAe?$AAm?$AA3?$AA2?$AA?2?$AAA?$AAs?$AAi?$AAB?$AAl?$AAC?$AAf?$AAg?$AA?4?$AAd@ 10006798     BluLinkCfg.obj
 0002:000007e8       ??_C@_17BIMEGBJF@?$AA2?$AA?0?$AA8?$AA?$AA@ 100067e8     BluLinkCfg.obj
 0002:000007f0       ??_C@_1CM@EGHHJIBM@?$AAA?$AAu?$AAd?$AAi?$AAo?$AAS?$AAc?$AAi?$AAe?$AAn?$AAc?$AAe?$AA?4?$AAA?$AAs?$AAi?$AAB?$AAl?$AAC?$AAf?$AAg?$AA?$AA@ 100067f0     BluLinkCfg.obj
 0002:00000820       ??_C@_1HC@EGCIGHEM@?$AAC?$AAo?$AAn?$AAf?$AAi?$AAg?$AAu?$AAr?$AAe?$AA?5?$AAB?$AAL?$AAU?$AA?5?$AAl?$AAi?$AAn?$AAk?$AA?5?$AAi?$AAn?$AAp?$AAu?$AAt?$AA?5?$AAa?$AAn?$AAd?$AA?5?$AAo?$AAu?$AAt@ 10006820     BluLinkCfg.obj
 0002:00000894       ??_C@_1CO@OMKBIMF@?$AAB?$AAL?$AAU?$AA?5?$AAl?$AAi?$AAn?$AAk?$AA?5?$AAC?$AAo?$AAn?$AAf?$AAi?$AAg?$AAu?$AAr?$AAa?$AAt?$AAi?$AAo?$AAn?$AA?$AA@ 10006894     BluLinkCfg.obj
 0002:000008c8       ??_C@_1EI@IPMPPGE@?$AAA?$AAu?$AAd?$AAi?$AAo?$AAS?$AAc?$AAi?$AAe?$AAn?$AAc?$AAe?$AA?5?$AAB?$AAL?$AAU?$AA?5?$AAl?$AAi?$AAn?$AAk?$AA?5?$AAC?$AAo?$AAn?$AAt?$AAr?$AAo?$AAl?$AA?5?$AAP?$AAa@ 100068c8     BluLinkCfg.obj
 0002:00000910       ??_C@_1EO@GGPFOMEM@?$AA?$HL?$AA7?$AAC?$AAC?$AAC?$AAF?$AA9?$AA7?$AA3?$AA?9?$AA9?$AA5?$AAF?$AA2?$AA?9?$AA4?$AAf?$AA5?$AAe?$AA?9?$AA8?$AA5?$AA7?$AA3?$AA?9?$AA9?$AA5?$AA3?$AA9?$AA3?$AAB?$AAD@ 10006910     BluLinkCfg.obj
 0002:00000960       ??_C@_1EA@LCPOBPC@?$AAN?$AAo?$AA?5?$AAB?$AAL?$AAU?$AA?5?$AAl?$AAi?$AAn?$AAk?$AA?5?$AAa?$AAd?$AAa?$AAp?$AAt?$AAe?$AAr?$AAs?$AA?5?$AAw?$AAe?$AAr?$AAe?$AA?5?$AAf?$AAo?$AAu?$AAn?$AAd?$AA?$AA@ 10006960     BluLinkCfg.obj
 0002:000009a0       ??_C@_0P@LKABJJMO@IsWow64Process?$AA@ 100069a0     BluLinkCfg.obj
 0002:000009b0       ??_C@_1BC@GDMECMAK@?$AAk?$AAe?$AAr?$AAn?$AAe?$AAl?$AA3?$AA2?$AA?$AA@ 100069b0     BluLinkCfg.obj
 0002:000009c8       ??_C@_1EK@CCCKMOMP@?$AAE?$AAr?$AAr?$AA?5?$AA?9?$AA?5?$AAm?$AAu?$AAl?$AAt?$AAi?$AAp?$AAl?$AAe?$AA?5?$AAK?$AAe?$AAy?$AAb?$AAo?$AAa?$AAr?$AAd?$AAH?$AAo?$AAo?$AAk?$AA?5?$AAo?$AAb?$AAj?$AAe@ 100069c8     ConfigDialog.obj
 0002:00000a18       ??_C@_1HM@MOHNHKHM@?$AAY?$AAo?$AAu?$AA?5?$AAm?$AAu?$AAs?$AAt?$AA?5?$AAr?$AAe?$AAb?$AAo?$AAo?$AAt?$AA?5?$AAy?$AAo?$AAu?$AAr?$AA?5?$AAc?$AAo?$AAm?$AAp?$AAu?$AAt?$AAe?$AAr?$AA?5?$AAf?$AAo@ 10006a18     ConfigDialog.obj
 0002:00000a98       ??_C@_1MK@ILLPMKJC@?$AAY?$AAo?$AAu?$AA?5?$AAm?$AAu?$AAs?$AAt?$AA?5?$AAr?$AAe?$AAb?$AAo?$AAo?$AAt?$AA?5?$AAy?$AAo?$AAu?$AAr?$AA?5?$AAc?$AAo?$AAm?$AAp?$AAu?$AAt?$AAe?$AAr?$AA?5?$AAt?$AAo@ 10006a98     ConfigDialog.obj
 0002:00000b68       ??_C@_1IK@MCLDGMBA@?$AAA?$AAd?$AAa?$AAp?$AAt?$AAe?$AAr?$AAs?$AA?5?$AAh?$AAa?$AAv?$AAe?$AA?5?$AAd?$AAi?$AAf?$AAf?$AAe?$AAr?$AAe?$AAn?$AAt?$AA?5?$AAs?$AAa?$AAm?$AAp?$AAl?$AAe?$AAr?$AAa@ 10006b68     ConfigDialog.obj
 0002:00000bf8       ??_C@_1LI@EINHHKMF@?$AAA?$AAd?$AAa?$AAp?$AAt?$AAe?$AAr?$AAs?$AA?5?$AAh?$AAa?$AAv?$AAe?$AA?5?$AAd?$AAi?$AAf?$AAf?$AAe?$AAr?$AAe?$AAn?$AAt?$AA?5?$AAW?$AAD?$AAM?$AA?5?$AAd?$AAe?$AAv?$AAi@ 10006bf8     ConfigDialog.obj
 0002:00000cb0       ??_C@_1GI@JONNNMHI@?$AAS?$AAo?$AAm?$AAe?$AA?5?$AAc?$AAh?$AAa?$AAn?$AAn?$AAe?$AAl?$AA?5?$AAs?$AAe?$AAt?$AAt?$AAi?$AAn?$AAg?$AAs?$AA?5?$AAn?$AAo?$AAt?$AA?5?$AAa?$AAp?$AAp?$AAl?$AAi?$AAe@ 10006cb0     ConfigDialog.obj
 0002:00000d18       ??_C@_15LNJDIFMI@?$AAI?$AAn?$AA?$AA@ 10006d18     ConfigDialog.obj
 0002:00000d20       ??_C@_17NFNCFLGO@?$AAO?$AAu?$AAt?$AA?$AA@ 10006d20     ConfigDialog.obj
 0002:00000d28       ??_C@_1DO@CFJJBDGO@?$AA?$CF?$AAd?$AA?5?$AA?9?$AA?5?$AAB?$AAL?$AAU?$AA?9?$AAP?$AAC?$AAI?$AA?5?$AAA?$AAS?$AAI?$AAO?$AA?5?$AA?$CF?$AAs?$AA?5?$AA?$CI?$AA?$CF?$AAd?$AA?5?$AA?9?$AA?5?$AA?$CF?$AAd?$AA?$CJ?$AA?$AA@ 10006d28     ConfigDialog.obj
 0002:00000d68       ??_C@_1EA@DMFCDEDA@?$AA?$CF?$AAd?$AA?5?$AA?9?$AA?5?$AAB?$AAL?$AAU?$AA?9?$AAP?$AAC?$AAI?$AA?1?$AA?$CF?$AAd?$AA?5?$AAW?$AAD?$AAM?$AA?5?$AA?$CF?$AAs?$AA?5?$AA?$CI?$AAd?$AAi?$AAr?$AAe?$AAc?$AAt?$AA?$CJ?$AA?$AA@ 10006d68     ConfigDialog.obj
 0002:00000da8       ??_C@_1CA@LANDJAEG@?$AAC?$AAh?$AAa?$AAn?$AAn?$AAe?$AAl?$AA?5?$AAN?$AAu?$AAm?$AAb?$AAe?$AAr?$AA?3?$AA?$AA@ 10006da8     ConfigDialog.obj
 0002:00000dc8       ??_C@_15OEEJMLKJ@?$AA4?$AA8?$AA?$AA@ 10006dc8     ConfigDialog.obj
 0002:00000dd0       ??_C@_15LIAIKPEE@?$AA9?$AA6?$AA?$AA@ 10006dd0     ConfigDialog.obj
 0002:00000dd8       ??_C@_13JGCMLPCH@?$AA1?$AA?$AA@ 10006dd8     ConfigDialog.obj
 0002:00000ddc       ??_C@_13IEJJBAMJ@?$AA2?$AA?$AA@ 10006ddc     ConfigDialog.obj
 0002:00000de0       ??_C@_13KBPCEPBF@?$AA4?$AA?$AA@ 10006de0     ConfigDialog.obj
 0002:00000de4       ??_C@_13OLCEPAKN@?$AA8?$AA?$AA@ 10006de4     ConfigDialog.obj
 0002:00000de8       ??_C@_1LA@FFMJMMLD@?$AAC?$AAh?$AAa?$AAn?$AAg?$AAe?$AAs?$AA?5?$AAc?$AAa?$AAn?$AAn?$AAo?$AAt?$AA?5?$AAb?$AAe?$AA?5?$AAa?$AAp?$AAp?$AAl?$AAi?$AAe?$AAd?$AA?5?$AAb?$AAe?$AAc?$AAa?$AAu?$AAs@ 10006de8     ConfigDialog.obj
 0002:00000e98       ??_C@_1CI@NKKEIBLI@?$AAS?$AAe?$AAS?$AAh?$AAu?$AAt?$AAd?$AAo?$AAw?$AAn?$AAP?$AAr?$AAi?$AAv?$AAi?$AAl?$AAe?$AAg?$AAe?$AA?$AA@ 10006e98     ConfigDialog.obj
 0002:00000ec0       ??_C@_17OMFOJHEJ@?$AAW?$AAT?$AAF?$AA?$AA@ 10006ec0     ConfigDialog.obj
 0002:00000ec8       __load_config_used         10006ec8     MSVCRT:loadcfg.obj
 0002:00000f10       ___safe_se_handler_table   10006f10     <linker-defined>
 0002:00000f18       ___rtc_iaa                 10006f18     MSVCRT:initsect.obj
 0002:00000f1c       ___rtc_izz                 10006f1c     MSVCRT:initsect.obj
 0002:00000f20       ___rtc_taa                 10006f20     MSVCRT:initsect.obj
 0002:00000f24       ___rtc_tzz                 10006f24     MSVCRT:initsect.obj
 0002:00001090       __IMPORT_DESCRIPTOR_COMCTL32 10007090     Comctl32:COMCTL32.dll
 0002:000010a4       __IMPORT_DESCRIPTOR_SETUPAPI 100070a4     Setupapi:SETUPAPI.dll
 0002:000010b8       __IMPORT_DESCRIPTOR_ASIHPI32 100070b8     asihpi32:ASIHPI32.dll
 0002:000010cc       __IMPORT_DESCRIPTOR_KERNEL32 100070cc     kernel32:KERNEL32.dll
 0002:000010e0       __IMPORT_DESCRIPTOR_USER32 100070e0     user32:USER32.dll
 0002:000010f4       __IMPORT_DESCRIPTOR_GDI32  100070f4     gdi32:GDI32.dll
 0002:00001108       __IMPORT_DESCRIPTOR_ADVAPI32 10007108     advapi32:ADVAPI32.dll
 0002:0000111c       __IMPORT_DESCRIPTOR_MSVCR120 1000711c     MSVCRT:MSVCR120.dll
 0002:00001130       __NULL_IMPORT_DESCRIPTOR   10007130     Comctl32:COMCTL32.dll
 0003:00000000       ___security_cookie         10008000     MSVCRT:gs_cookie.obj
 0003:00000004       ___security_cookie_complement 10008004     MSVCRT:gs_cookie.obj
 0003:00000010       ___native_dllmain_reason   10008010     MSVCRT:natstart.obj
 0003:00000838       ?__type_info_root_node@@3U__type_info_node@@A 10008838     MSVCRT:tncleanup.obj
 0003:00000840       ?g_phSubSys@@3PAUhpi_hsubsys@@A 10008840     AdapterInfo.obj
 0003:00000844       ?hinstance@@3PAUHINSTANCE__@@A 10008844     BluLinkCfg.obj
 0003:00000848       ?hYellowBrush@@3PAUHBRUSH__@@A 10008848     ChanControl.obj
 0003:0000084c       ?hGreenBrush@@3PAUHBRUSH__@@A 1000884c     ChanControl.obj
 0003:00000850       ?hRedBrush@@3PAUHBRUSH__@@A 10008850     ChanControl.obj
 0003:00000854       ?m_focus@KeyboardHook@@0_NA 10008854     ConfigDialog.obj
 0003:00000858       ?szTitle@@3PA_WA           10008858     ConfigDialog.obj
 0003:00000920       ?m_hkbhook@KeyboardHook@@0PAUHHOOK__@@A 10008920     ConfigDialog.obj
 0003:00000928       ___@@_PchSym_@00@UzhrUhdUzkkhUyoformpxutUivovzhvUhgwzucOlyq@850942038A092919 10008928     stdafx.obj
 0003:0000092c       ___native_startup_lock     1000892c     <common>
 0003:00000930       ___native_startup_state    10008930     <common>
 0003:00000934       ___onexitend               10008934     <common>
 0003:00000938       ___onexitbegin             10008938     <common>
 0003:0000093c       ___dyn_tls_init_callback   1000893c     <common>

 entry point at        0001:00003f58

 Static symbols

 0001:00001fe4       $LN31                      10002fe4     * CIL library *:* CIL module *
 0001:00001ff4       $LN28                      10002ff4     * CIL library *:* CIL module *
 0001:000020f0       _swprintf                  100030f0 f   * CIL library *:* CIL module *
 0001:000020f0       _swprintf                  100030f0 f   * CIL library *:* CIL module *
 0001:00002fd8       $LN28                      10003fd8     * CIL library *:* CIL module *
 0001:000034b8       $LN158                     100044b8     * CIL library *:* CIL module *
 0001:00003d15       _pre_c_init                10004d15 f   MSVCRT:crtdll.obj
 0001:00003f7b       ___DllMainCRTStartup       10004f7b f   MSVCRT:crtdll.obj
 0001:00004530       $$000000                   10005530     MSVCRT:sehprolg4.obj
 0001:00004600       __unwindfunclet$?RunDialog@@YAXPAUHWND__@@_N@Z$0 10005600 f   * CIL library *:* CIL module *
 0001:00004608       __unwindfunclet$?RunDialog@@YAXPAUHWND__@@_N@Z$1 10005608 f   * CIL library *:* CIL module *
 0001:00004610       __ehhandler$?RunDialog@@YAXPAUHWND__@@_N@Z 10005610 f   * CIL library *:* CIL module *
 0002:000001fc       _pcinit                    100061fc     MSVCRT:crtdll.obj
 0002:00000200       _pinit                     10006200     MSVCRT:atonexit.obj
 0002:0000021c       _GS_ExceptionPointers      1000621c     MSVCRT:gs_report.obj
 0002:000004d0       _dwOne                     100064d0     * CIL library *:* CIL module *
 0002:00000f28       __unwindtable$?RunDialog@@YAXPAUHWND__@@_N@Z 10006f28     * CIL library *:* CIL module *
 0002:00000f38       __ehfuncinfo$?RunDialog@@YAXPAUHWND__@@_N@Z 10006f38     * CIL library *:* CIL module *
 0002:00000f60       __sehtable$___DllMainCRTStartup 10006f60     MSVCRT:crtdll.obj
 0002:00000f88       __sehtable$__IsNonwritableInCurrentImage 10006f88     MSVCRT:pesect.obj
 0002:00000fa8       __sehtable$__onexit        10006fa8     MSVCRT:atonexit.obj
 0002:00000fd0       .edata                     10006fd0     AsiBlCfg.exp
 0002:00000ff8       rgpv                       10006ff8     AsiBlCfg.exp
 0002:00001008       rgszName                   10007008     AsiBlCfg.exp
 0002:00001018       rgwOrd                     10007018     AsiBlCfg.exp
 0002:00001020       szName                     10007020     AsiBlCfg.exp
 0002:0000102d       $N00001                    1000702d     AsiBlCfg.exp
 0002:0000103f       $N00002                    1000703f     AsiBlCfg.exp
 0002:00001053       $N00003                    10007053     AsiBlCfg.exp
 0002:00001075       $N00004                    10007075     AsiBlCfg.exp
 0002:00001334       .idata$6                   10007334     Comctl32:COMCTL32.dll
 0002:000013aa       .idata$6                   100073aa     Setupapi:SETUPAPI.dll
 0002:0000159c       .idata$6                   1000759c     asihpi32:ASIHPI32.dll
 0002:00001642       .idata$6                   10007642     kernel32:KERNEL32.dll
 0002:000018a2       .idata$6                   100078a2     user32:USER32.dll
 0002:00001914       .idata$6                   10007914     gdi32:GDI32.dll
 0002:000019ea       .idata$6                   100079ea     advapi32:ADVAPI32.dll
 0002:00001a4a       .idata$6                   10007a4a     MSVCRT:MSVCR120.dll
 0003:00000018       _ClassesEntrySubList2      10008018     * CIL library *:* CIL module *
 0003:0000007c       _ControlPanelNamespaceRegList 1000807c     * CIL library *:* CIL module *
 0003:00000088       _ClassesEntryList          10008088     * CIL library *:* CIL module *
 0003:0000013c       _ControlPanelNamespaceEntryList 1000813c     * CIL library *:* CIL module *
 0003:00000178       _ClassesRegList            10008178     * CIL library *:* CIL module *
 0003:00000184       _ClassesEntrySubList1      10008184     * CIL library *:* CIL module *
 0003:000001c0       _PolicyRegList             100081c0     * CIL library *:* CIL module *
 0003:000001d0       _PolicyEntryList           100081d0     * CIL library *:* CIL module *
 0003:00000220       _originalDialogResource    10008220     * CIL library *:* CIL module *
 0003:00000510       ___proc_attached           10008510     MSVCRT:crtdll.obj
 0003:00000518       _GS_ExceptionRecord        10008518     MSVCRT:gs_report.obj
 0003:00000568       _GS_ContextRecord          10008568     MSVCRT:gs_report.obj
 0003:00000834       _DebuggerWasPresent        10008834     MSVCRT:gs_report.obj
 0003:00000924       ?pScrollbar@?1??DialogProc@@YGHPAUHWND__@@IIJ@Z@4PAVAsiScrollbar@@A 10008924     * CIL library *:* CIL module *
 0004:000002d0       $R000000                   100092d0     BluLinkCfg.res
 0004:00000f78       $R000CA8                   10009f78     BluLinkCfg.res
 0004:00000f90       $R000CC0                   10009f90     BluLinkCfg.res
 0004:00000fe0       $R000D10                   10009fe0     BluLinkCfg.res
 0004:00000ff0       $R000D20                   10009ff0     BluLinkCfg.res
 0004:00001108       $R000E38                   1000a108     BluLinkCfg.res
 0004:00001478       $R0011A8                   1000a478     BluLinkCfg.res
 0004:0002c920       $R02C650                   10035920     BluLinkCfg.res
 0004:0002cc70       $R02C9A0                   10035c70     BluLinkCfg.res
 0004:0002ccd8       $R02CA08                   10035cd8     BluLinkCfg.res
